:020000020000FC
:10000000F2C009C009C009C009C057C057C058C0D4
:10001000C9C0E8C054C0189518951895CF93DF93C0
:100020001F922F921F931FB71F9365FBA6F563FBCB
:10003000BEF410B316FBA6F4109074001394109243
:10004000740013E0111661F4677FF0927200F09271
:100050007300F09274001091A60012601093A60035
:10006000C0917200D0917300209769F419B71F7B7B
:1000700019BF1FB51F731FBDC69A1091A6001E7F22
:100080001093A60012C016B313FB2EF02197C09355
:100090007200D09373001AB510906000110E1BB55A
:1000A00020906100211E2BBC1ABC1F911FBF1F9105
:1000B0002F901F90DF91CF9118951895189518954E
:1000C0002F933F930F92AF93BF93EF93FF931F92A2
:1000D0002F923F921F931FB71F9322E61BB114FB71
:1000E00076F910FB2EF01CB1312E77FB36F011C0E3
:1000F0001CB1312E1AB111FB66F010907100112065
:1001000009F442C010906D0020906E00121834F176
:1001100032C010919F001F71232C269426942694A0
:10012000211A31F0F0927100F0926D0078682CC0C5
:100130007068777F1AE0109375001FEF10937100BD
:10014000F0926D0017E03122E4E4F1E08894EE1FB4
:10015000FF1FE30DFF1DC89500926E0030916D00EA
:10016000230FBB27A22F3C92339530936D001AE0EA
:100170001093750009C030916D00230FBB27A22F8B
:100180003C921FEF109370001F911FBF1F913F9073
:100190002F901F90FF91EF91BF91AF910F903F91E2
:1001A0002F911895AF93BF931F931FB71F93109173
:1001B0006F00139510936F00155041F0A8E6109151
:1001C0006F00A10FBB271C911CB906C0539855980E
:1001D000F0926A00F0926B001F911FBF1F91BF91B8
:1001E000AF91189518951FED1DBFFF24A0E6B0E054
:1001F000FD9219ED1A1BE1F71FE015BF10E01BBFC0
:1002000010E019BF12E013BF10E41FBD13E41EBDC0
:10021000A89518E011BD112718BB12BB1CEF17BB26
:100220001CE311BB14E91AB91CE019B913E018B9A1
:100230002FD0A8D1DED101D27894DD24F2BE8CE794
:1002400092B79817EAF31CE7810FE8E3F1E013E0B7
:10025000D122ED2C8894EE1C8894EE1FFF1FEE0D2A
:10026000FF1DC895E8E3F1E0E00DFF1DD39409946C
:100270000400060008000A0039D0E2CF84D1E0CFA4
:10028000B9D1DECFDBD1DCCF0305020101010302CE
:1002900077276627C59AC49AC69A28E03327AEE91D
:1002A000B0E01CB310FBEEF33EBB11E01CBB1DB372
:1002B0001D9333952A952223A1F71091A5001F7055
:1002C000110F110F22B3207F212322BB16B310FB85
:1002D00070F90EF0529811FB2EF017E619B9F09252
:1002E0009F00089510919E0019B908951090700014
:1002F000112009F41AC1F0927000EEE8F1E01090BC
:1003000062008894111C8894EE1FFF1FE10DFF1DF1
:10031000C895EEE8F1E0E00DFF1D099408004000EB
:1003200064008D009700B600B700D5006F7D109176
:10033000A60015601093A600F092A700F092A80006
:100340000BD124FB96F01091A6001B7F1093A60002
:10035000109164001093610010916500109360008B
:1003600010E010937900E3D0DFC010916400109387
:10037000780010916500109377001091A3001093FE
:1003800061001091A400109360001091A2001093DE
:100390007A0011E010937900CAD0C6C010916300B2
:1003A00013FB63F9F0927400D7D0F092A700F0929B
:1003B000A80060621091A60011601D7F1093A60036
:1003C00010916600109373001091670010937200F3
:1003D000109164001093610010916500109360000B
:1003E000A6D0A2C01091A60014601093A600606170
:1003F0001091A60010FB0EF097C03091630030936F
:100400007800209164002093770040916000509123
:100410006100421B530B38F0452B442339F011E0A7
:100420001093790003C012E0109379001091A2009C
:1004300010937A0079C0109163001F70110F110F93
:1004400022B3237C212B22BB6FC06B7E20916300E3
:1004500021FB5EF41FEF109377001093780012E0F9
:100460001093790020FB62F95FC01091A6001E7FF7
:100470001093A60020FB0EF0C69A1FB51F731FBD78
:1004800019B71F7B19BF50C04FC01091630010FBFC
:1004900056F0A0EAB0E010916400A10FBF1D1091CA
:1004A00065001C9341C01CB311FBEEF31091640076
:1004B0001EBB109165001DBBF89414E01CBB12E03C
:1004C0001CBB789431C01091630010FBFEF011FB4F
:1004D00066F0A0EAB0E010916400A10FBF1DF09299
:1004E0006A001C9110936B001FC0A0EAB0E010914D
:1004F0006400A10FBF1D1D912C913E91311B332330
:10050000A1F710936A0020936B000EC01CB310FB80
:10051000EEF3109164001EBB11E01CBB2DB3F092F2
:100520006A0020936B0000C07460A895089519B705
:100530001F7B19BF1CB510906000110E1DB52090D7
:100540006100211E2BBC1ABC18B7106418BF19B764
:10055000106419BFC6980895F8941FB51F731064EE
:100560001FBD1EB51C7F2091630023952370122BA5
:100570001EBD78942091630022FB66F918B312F92E
:1005800018BB0895089577FB0EF031C0579872FBA1
:100590002EF4737710919F0010680DC020917500A4
:1005A0002A952093750019F573FB77770EF41FC019
:1005B00010919F001F7776FB16F910936800F09258
:1005C0007100F0926D001091680020916900120F87
:1005D00020916A00120F20916B00120F10936C0093
:1005E000F0926F0010916800539A1CB9559A579A6F
:1005F0000895089550907600552009F41DC0ACE18F
:10060000AB5150906300A51918F4F092760014C015
:10061000F0927600EBE1F3E0509063008894551C73
:100620008894EE1FFF1FE50DFF1DC895EBE1F3E079
:10063000E00DFF1D099401000895089510917A00BE
:10064000112321F01A9510937A007FC0A1E4AE53D4
:1006500070907900A71908F478C0EEE3F3E0709089
:1006600079008894771C8894EE1FFF1FE70DFF1D0B
:10067000C895EEE3F3E0E00DFF1D099403000400CC
:100680002D0063C01091A20010937A0020916000A9
:10069000309161004091A1005091A000241B350BC6
:1006A00038F04091770050917800421B530B60F076
:1006B000209177003091780010E01093790010912C
:1006C000A6001B7F1093A600F8942093600030933F
:1006D000610078943AC01091A20010937A002091A2
:1006E0006000309161004091A1005091A000240F62
:1006F000351F38F04091770050917800421B530B22
:10070000F0F410E01093790064FB56F42091770028
:10071000309178001091A6001B7F1093A6000FC0A7
:100720001091A6001E7F1093A60019B71F7B19BF5A
:1007300062FB5EF0C69A1FB51F731FBD06C0F8941A
:0C074000209360003093610078940895CD
:00000001FF
